:020000040000FA
:100000000508A2000608A3001D288312C800CE011F
:100010001828831203131630A0002C30A1000A12F6
:100020008A11A10B0F280A128A11A00B0D28CE0AE3
:100030004E084802031D09280800BC014414C410DE
:100040004411C4159328C800613048024E10031DA6
:1000500003184E147A304802CE10031D031CCE1430
:100060004E154E18CE1C4E114E1D3828E030C807D4
:1000700048080800C8004808BF3E0318F93E113E72
:10008000C80048080800EC006C08F63E0318073E5C
:100090003A3EEC006C0808008312E600E70179287C
:1000A0002808A7002908A8002A08A9002B08AA00E8
:1000B0002C08AB002D08AC002E08AD002F08AE00B8
:1000C0003008AF003108B0003208B1003308B20088
:1000D0003408B3003508B4003608B5003708B60058
:1000E0003808B7003908B8003A08B9003B08BA0028
:1000F000E70A67086602031D5028080083124416A9
:1001000022122208850008008312441222162208B7
:1001100085000800C412441AC41608008312C41EC5
:1001200092287E28842844138A15792D44199F2803
:10013000831606108312C41D9F288316861183120E
:100140002215220885004417080083160614861518
:100150008312221122088500441308008312231001
:10016000C41B231423088600C41FB828C413B9284D
:10017000C417A311C41BA31523088600080083120B
:100180002310C41B231423088600C41FC928C413CA
:10019000CA28C417A311C41BA31523088600000096
:1001A00000000000000008008316A0008312EF0189
:1001B000E628A201BF208A11BF208316A20A0A30B6
:1001C00022028A11031DDA288312EF0A6F088316B0
:1001D0002002031DD92808008312EE008316A00117
:1001E000FE28EF01BF208A11BF208312EF0A64307E
:1001F0006F028A11031DF2288316A00A20088312B9
:100200006E02031DF12808006E1C0A29EE10441826
:10021000EE140D29EE10C418EE148A208A118420E1
:1002200083126E156E18441D6E11A3136E19A31759
:10023000230886008316861383122313EE182317D0
:1002400023088600831606138312A211EE18A21546
:1002500022088500A2142208850032308A11D42099
:100260008312A2102208850032308A11D42083160E
:10027000861706178312A2112208850032308A11D0
:10028000D4208A118E28441F49290A30EC208A1173
:100290004D299620C8308A11EC208312A21422081E
:1002A0008500221022088500A312230886008316E9
:1002B0000510861283126E148A1104298316051400
:1002C00086168312A21422088500441F6B29A520DC
:1002D000C8308A11EC2083126E106D186E148A11CA
:1002E000042983126D105E2983126D145E29831216
:1002F000E60024308316980083126608831699005E
:100300009030831298008316861406110800831615
:10031000861406118312231523088600831698017C
:100320009901831298010800831220100C1A2014DE
:100330000800E600942183126710201867148A11C0
:100340006718A529AE208A119A2966089900080025
:1003500083129810181DB1298618AF29AC29403096
:100360007721831220108C1A201408001A08080024
:100370008316A4008612A601D5292418C229831247
:10038000A312C4298312A31623088600221422086C
:10039000850003108316A40CAE20831222102208BD
:1003A00085008A11AE208316A60A260825028A1126
:1003B000031DBD29BF288312EC0083168616831205
:1003C000EE01F329221422088500AE2003108312C7
:1003D000ED0CED13861AED172210220885008A1104
:1003E000AE208312EE0A6E086C028A11031DE22908
:1003F000BF2083126C098316A0000930A0072008D3
:10040000FE0083126D088316A100FE088A110319ED
:100410000D2A0310A10CFE0B092A210808008312E3
:10042000E7006708DB218312E8000F306805E90068
:1004300069088A1143288312ED0006308316A5004F
:1004400083126D08B829ED0001308316A500003035
:10045000B82108308316A50083126E088A11B821CE
:1004600006308316A50083126D088A11B821013069
:100470008316A50000308A11B8298312EF000430DA
:100480008316A50083126F08B82108308316A500D3
:1004900023088A11B82108308316A50022088A1182
:1004A000B8298312E60004308316A500831266087B
:1004B000B82108308A11DB2108308A11DB2903308A
:1004C0008316A5000030B8218312A31223088600EA
:1004D0002214220885003D088A11D420831222109C
:1004E000220885008A11BF2010308316A500003035
:1004F0008A11B8290E308316A20083124108831690
:10050000A30000303D226E308316A200F830A30015
:1005100000308A113D220E308316A200831240085B
:100520008316A30000308A113D226E308316A2008C
:10053000F730A30000308A113D220E308316A2004E
:1005400083123F088316A30000308A113D226E30CB
:100550008316A200F630A30000308A113D2A8312D0
:10056000E700E801C02AAE208312BF0A3F088A11C3
:10057000031DBF2AC00A4008031DBF2AC10AE80A9A
:1005800068086702031DB32A08008312ED006D0896
:10059000C1006E08C000831620088312BF007A2AAB
:1005A0008E308316A200A630A30000303D228C308E
:1005B0008316A200A630A30000308A113D228312C8
:1005C000EE0106308316A0003C308A11C522831646
:1005D000A201A3010C308A113D2A7E208312250836
:1005E000A600BC010130BE00380EF039CE004E0826
:1005F0003907BD00C101C001BF010A303B028A11A9
:10060000031D052B84208A1174290B303B02031D26
:10061000162B4410BA184414C4103A19C4144411C7
:100620003A184415C411BA19C41508000C303B021D
:10063000031DDC2B3A08CF15031DCF1105303A02FC
:100640004F1203194F16CF12CF1D4F1ACF16CF1EC0
:10065000372B0130BC006430C800432105308312C1
:100660003A028A11031D9B2E0430BE009B2E0130DE
:100670003A02031D422B0330BC000A30C80043215C
:100680008A119B2E02303A02031D4D2B0530BC000F
:100690000A30C80043218A119B2E03303A02D01041
:1006A0000319D01406303A02501103195015D01115
:1006B000D01C5019D01509303A02501203195016A7
:1006C000D012D01D501AD016D01E8D2B3230BC0047
:1006D0000A30C80043218A11D0228E308316A2002E
:1006E000A630A30000308A113D229C308316A20060
:1006F000A630A30000308A113D228312EE0183163A
:10070000A00100308A11C522063083123A028A11F4
:10071000031DDB2B0830BE009B2E04303A02031D64
:10072000982B0130BC005030C80043218A119B2E09
:1007300007303A0251100319511408303A02D1100F
:100740000319D1145111511CD1185115511DB52B3C
:100750003A08BC000A30C80008303A02031DB22B28
:100760001E30C80043218A119B2E0B303A02031D14
:10077000C02B0930BC001430C80043218A119B2EC5
:100780000A303A02031DCE2B0B30BC001430C800D7
:10079000432106308A111B228A119B2E0C303A020B
:1007A000031DD92B0C30BC001930C80043218A111D
:1007B0009B2E3F30A6009B2E0D303B02031D722C5A
:1007C0002130C0003A085214031D521008303A027A
:1007D000D2100319D2145211521CD2185215521DA4
:1007E000F82B0230BC006430C80043218A119B2ED4
:1007F00001303A02031D032C0430BC006430C800F1
:1008000043218A119B2E02303A02521203195216CA
:1008100007303A02D2120319D2165213521ED21ABC
:100820005217521F1A2C0630BC006430C8004321F6
:100830008A119B2E0C303A02031D252C0D30BC0072
:100840006430C80043218A119B2E03303A025310B2
:100850000319531406303A02D3100319D314531159
:10086000531CD318531509303A02D3110319D31569
:100870005312531DD3195316531E642C3330BC002E
:100880000A30C80043218312C0019E308316A200A3
:10089000A630A30000308A113D229C308316A200AE
:1008A000A630A30000308A113D22063083123A029E
:1008B0008A11031D5D2C0830BE0009303A02031D69
:1008C000712C3530BC009B2E04303A02031D6F2C76
:1008D0005030C8000230BC0043218A119B2E3F30AB
:1008E000A6009B2E0F303B02031D432D2030C0007D
:1008F0003A08D414031DD41001303A0254110319DC
:100900005415D411D41C5419D41502303A0254127F
:1009100003195416D412D41D541AD41604303A02B2
:10092000541303195417D413D41E541BD41707306F
:100930003A02551003195514D510D41F5518D51463
:1009400008303A02551103195515D511D51C551902
:10095000D5150B303A02551203195516D512D51D6F
:10096000551AD5160C303A02551303195517D513DD
:10097000D51E551BD517D51FF72C0130BC004321C0
:1009800000308A111B228312EE0100308A112322CB
:1009900064308312C80002303A025610031956140C
:1009A00007303A02D6100319D6145611561CD61821
:1009B00056158A11561DDE2C0530BC0001303A0256
:1009C000D6110319D6150B303A02561203195616D2
:1009D000D612D61D561AD616D61EF02C0330BC00E1
:1009E0000C303A02031D9B2E0C30BC009B2E0330B2
:1009F0003A02D6130319D61706303A0257100319D4
:100A00005714D710D61F5718D71409303A02571168
:100A100003195715D711D71C5719D715D71D352DC1
:100A20003430BC0043218E308316A200A630A300D0
:100A300000308A113D228C308316A200A630A3001C
:100A400000308A113D228312EE018316A00130305E
:100A50008A11C5220A308312C80006303A028A1170
:100A6000031D9B2E0830BE009B2E0A303A02031D48
:100A7000402D0B30BC001430C80043218A119B2E3E
:100A80003F30A6009B2E0E303B02031D992E3A08E4
:100A9000031D8F2D432100308A111B22FF3083124A
:100AA000EE003F308A1123228312EC0106308A11B6
:100AB0001B228312EC0A07306C028A11031D562D8B
:100AC00001301B2207308A111B2208308A111B2299
:100AD0000A308A11EC2001308A111B2207308A115A
:100AE0001B2283126E148A11042103308A111B22E7
:100AF000FF308312EE0000308A11232208308A1161
:100B00001B220A308A11EC200B308A111B2208307C
:100B10008A111B220A308A11EC208A119B2E013087
:100B20003A02031DA42D432100308A111B22831297
:100B3000EE0100308A11232209308A111B2228304D
:100B40008A11EC208A119B2E02303A0258110319A7
:100B5000581507303A02D8110319D8155812581DE4
:100B6000D8195816581EC52D432100308A111B2252
:100B70008312EE0100308A1123221F308A111B22BA
:100B800005308A11EC208A119B2E04303A02D812CB
:100B90000319D8160B303A02581303195817D813F3
:100BA000D81E581BD817D81FED2D432100308A11AD
:100BB0001B22FF308312EE003F308A1123220930BE
:100BC0008A111B220A308A11EC200B308A111B2259
:100BD0000A308A11EC208A119B2E08303A02031D3C
:100BE0000F2E432100308A111B22FF308312EE00AA
:100BF0003F308A11232209308A111B220A308A11C0
:100C0000EC2009308A111B220A308A11EC200B30AB
:100C10008A111B220A308A11EC208A119B2E0C307B
:100C20003A02031D222E432109308A111B2206306D
:100C30008A11EC200B308A111B2206308A11EC201D
:100C40008A119B2E03303A02031D4D2E432183123D
:100C5000EE0104308316A0003C308A11C5228316B1
:100C6000A2018030A3000C308A113D228316A2011C
:100C7000A30100308A113D2204308316A500003004
:100C80008A11B82106308A11EC2010308316A50095
:100C900000308A11B8218A119B2E09303A02031DB7
:100CA000892E43218312EE0105308316A0003C30CB
:100CB0008A11C5223F308316A2003F30A3000C30BA
:100CC0008A113D228312EE0104308316A0003C30CD
:100CD0008A11C5228F308316A2008F30A3000C30FA
:100CE0008A113D228316A201A30100308A113D2200
:100CF00004308316A50000308A11B82106308A110D
:100D0000EC2010308316A50000308A11B8218A111A
:100D10009B2E0A303A02031D962E432109308A1178
:100D20001B2214308A11EC208A119B2E3F30A60022
:100D30009B2E3F30A60083123D08031DA12E4808BC
:100D4000BD00080032303C020319AF2E0318AF2E4D
:100D50002508A60006301B2201308A11AF2A3F3039
:100D6000A6000800E60066081B2201308A11DB217C
:100D700004308A110F228312BB0004308A110F2223
:100D80008312BA0004308A110F228312B900023094
:100D90008A110F228312B80001308A11DB2910302A
:100DA000C8002508A60032303C020319D92E031CC6
:100DB000DB2E1230C800CE018A150F2801303C020C
:100DC000DA100319DA1403303C025A1103195A15C8
:100DD000DA11DA1C5A19DA1505303C025A120319D5
:100DE0005A16DA12DA1D5A1ADA1607303C025A136A
:100DF00003195A17DA13DA1E5A1BDA1709303C02A4
:100E00005B1003195B14DB10DA1F5B18DB140B306B
:100E10003C025B1103195B15DB11DB1C5B19DB1555
:100E20000C303C025B1203195B16DB12DB1D5B1AF4
:100E3000DB16DB1E2E2F0430B226013083123E0259
:100E40008A110319262F031C262FA22604308A118B
:100E50004C2004308312C8028A150E2802303C024E
:100E6000DB130319DB1704303C025C1003195C141C
:100E7000DC10DB1F5C18DC1406303C025C1103192B
:100E80005C15DC11DC1C5C19DC150D303C025C12BD
:100E900003195C16DC12DC1D5C1ADC16DC1E5F2FED
:100EA0000530B22630308312B8003030B90004303B
:100EB0008A114C2004308312C8028A150E28323061
:100EC0003C025C1303195C1734303C02DC13031939
:100ED000DC175D105C1FDC1B5D145D1C8E2F093060
:100EE00051228312E500650E0F39CF004F088A1199
:100EF00043208312BA000F306505CF004F088A11D6
:100F000043208312BB0001308A11AF2202308A11C4
:100F10004C2002308312C8028A150E2833303C025E
:100F2000DD100319DD1435303C025D1103195D1528
:100F3000DD11DD1C5D19DD158A15DD1D0C280E3057
:100F40008316A20083123F088316A30000308A1183
:100F50003D226E308316A200A930A30000308A1112
:100F60003D220E308316A200831240088316A30090
:100F700000308A113D226E308316A200AA30A300F1
:100F800000308A113D2280308316A200A630A300D3
:100F900000308A113D2250308316A200A830A300F1
:100FA00000308A113D226E308316A200F530A30076
:100FB00000308A113D22353083123C028A11031D14
:100FC000EC2F8316A201A30100303D228316A2015B
:100FD000A30100308A113D2202308A11512283126E
:100FE000E500650E0F39CF004F088A1143208312A8
:100FF000BA000F306505CF004F088A1143208312D5
:10100000BB0001308A11AF2202308A114C2002301D
:101010008312C8028A150E283F30A600CE0A4E0859
:101020003E028A11031DDE2E48084C28E70067089F
:101030008A111B2201308316A50000308A11B821C5
:1010400004308316A50083123B088A11B8210430AE
:101050008316A50083123A088A11B821043083163A
:10106000A500831239088A11B82102308316A50021
:10107000831238088A11B82101308316A500003088
:101080008A11B821831268088A111B2283123D0835
:101090008A11D42083126B088A15031952286B0811
:1010A0008A111B2A08008A117E2083122508A600B7
:1010B00001303C028A15031D62280830E800EB016C
:1010C0000230162802303C02031D6B280830E8006D
:1010D000EB010330162803303C02031D752808304D
:1010E000E8000E30EB000230162804303C02031DED
:1010F0007C283F30A600080005303C02031D8628EE
:101100001830E8001730EB000230162806303C0299
:10111000031D90281830E8001730EB000330162824
:101120000D303C02031D9A281830E8000A30EB000D
:101130000330162807303C02DE130319DE1708308F
:101140003C025F1003195F14DF10DE1F5F18DF140D
:1011500009303C025F1103195F15DF11DF1C5F19B5
:10116000DF15DF1D2E290430E60066080319072964
:10117000E60302308A111B2201308316A5000030DD
:101180008A11B82104308316A50083122F088A1112
:10119000B82104308316A50083122E088A11B821C5
:1011A00004308316A50083122D088A11B82102305D
:1011B0008316A50083122C088A11B82101308316EA
:1011C000A50000308A11B821831266088A15031918
:1011D000EC2806308A111B2283123008AC00340838
:1011E000B0003808B4003108AD003508B100390846
:1011F000B5003208AE003608B2003A08B60033082F
:10120000AF003708B3003B08B7008A15B52818307F
:101210008A111B2283123D088A11D42007308312C1
:101220003C028A15031D192917308A111B228A15C1
:10123000282908303C02031D22290A308A111B226A
:101240008A1528290E308A111B2202308A11D420D7
:1012500006308A111B2204308A11AF2A08303C0262
:10126000031D38290830E8000E30EB000230162844
:101270000C303C02031D41290830E800EB0102302C
:1012800016280B303C02031D4B290830E8000E30B5
:10129000EB000230162832303C02031DB2298A11BD
:1012A0007A2283122E0EF039C8002F084807C90091
:1012B0002C0EF039CA002D084A07CB0049088316C6
:1012C000A20083124B088316A3000D308A113D2221
:1012D0008312320EF039C80033084807C900300EB7
:1012E000F039CA0031084A07CB0049088316A2002A
:1012F00083124B088316A3000D308A113D228312FE
:10130000360EF039C80037084807C900340EF039E6
:10131000CA0035084A07CB0049088316A200831289
:101320004B088316A3000D308A113D2283123A0E1A
:10133000F039C8003B084807C900380EF039CA0028
:1013400039084A07CB0049088316A20083124B08CC
:101350008316A3000F308A113D228A115F220830C4
:101360008A11AF2A33303C026012031960163530FF
:101370003C02E0120319E0166013601EE01A6017C9
:10138000601F6B2A0E308316A20083123F0883165B
:10139000A30000308A113D226E308316A200A930CE
:1013A000A30000308A113D220E308316A200831262
:1013B00040088316A30000308A113D226E30831648
:1013C000A200AA30A30000308A113D2283123A0EF7
:1013D000F039C8003B084807C9000E308316A20048
:1013E000831249088316A30000308A113D226E3013
:1013F0008316A200A830A30000308A113D22843059
:101400008316A200A630A30000308A113D2233309B
:1014100083123C028A15031D2D2A0E308316A2006A
:101420005530A30000308A113D226E308316A20091
:10143000A730A30000308A113D220E308316A2008F
:10144000AA30A30000308A113D226E308316A2001C
:10145000A730A30000308A113D2282308316A200FB
:10146000A630A30000308A113D2250308316A2001E
:10147000A630A30000308A113D226E308316A200F0
:10148000F530A30000308A113D22353083123C0232
:101490008A15031D512A8316A201A30100308A1167
:1014A0003D2204308316A50002308A11B82106308F
:1014B0008A11EC2010308316A50000308A11B82163
:1014C00094308316A200A630A30000308A113D227A
:1014D00001308A11AF2A34303C02031D872A8A1159
:1014E0007A2283123A0EF039C8003B084807E6001A
:1014F00066088316A200831266088316A3000F30C5
:101500008A113D228A115F2201308A11AF2A3F30B1
:10151000A600080053282508A60032303C02031913
:10152000C32A0318C32A8312360EF039C8003708BD
:101530004807C90041084902E310031DE314380EAF
:10154000F039CA0039084A07CB0040084B02631142
:10155000031D6315E311E31C6319E3153A0EF0391B
:10156000CC003B084C07CD003F084D026312031D21
:101570006316E312E31D631AE316E31E022B8A11BE
:10158000A2268A15932A32303C026313031963178B
:1015900033303C02E3130319E3176410631FE31BAA
:1015A000641434303C02E4100319E4146411641C24
:1015B000E418641535303C02E4110319E415641293
:1015C000641DE4196416641E002B360EF039C80041
:1015D00037084807C900380EF039CA0039084A07E9
:1015E000CB003A0EF039CC003B084C07CD004B083D
:1015F000EE004D088316A000831249088A11C52AFF
:101600003F30A60008008A1187218A1171298316AC
:10161000861605108312861C0F2B6810102B681479
:1016200022106818221422088500861E192BE81043
:101630001A2BE8142311E8182315230886008618AE
:10164000E7016608031D2A2BE70A1E306702031D07
:101650002A2B0800E60A0A2B831686160510831229
:10166000221086182214220885002311861A2315B9
:10167000230886008618E7016608031D452BE70A44
:101680001E306702031D452B0800E60A2F2B831628
:10169000061306168312861C4F2B6810502B6814F5
:1016A00023136818231723088600061E592BE810F9
:1016B0005A2BE8142311E8182315230886008618EE
:1016C000E7016608031D6A2BE70A1E306702031D47
:1016D0006A2B0800E60A4A2B8316061306168312A5
:1016E000231386182317230886002311061A2315AF
:1016F000230886008618E7016608031D852BE70A84
:101700001E306702031D852B0800E60A6F2B8A1125
:10171000842083123B088A15031D932B03238A150B
:1017200007238A15382D01303B02031D9C2B032310
:101730008A152C238A15382D02303B02031DA52B58
:1017400003238A1547238A15382D03303B02031DD6
:10175000AE2B03238A156C238A15382D04303B02E7
:10176000031DDF2B25088A11992114308A11EC20E2
:1017700083123A088A15031DC02B81308A117729FC
:1017800001303A02031DC72B40308A1177290230FD
:101790003A02031DCE2B20308A11772903303A02FA
:1017A000031DD52B15308A11772904303A02031D09
:1017B000DC2B0A308A1177293F30A600080005305B
:1017C0003B0249110319491506303B02C91103199F
:1017D000C9154912491DC919491607303B02C912DA
:1017E0000319C9164913491EC91A4917491FEF2C75
:1017F0004B1005303B0203194B1406303B02CB1053
:101800000319CB143A1C112C4B18092C8316051004
:101810000B2C8316051483122210CB1822142208D5
:101820008500BA1C202C4B18182C831685101A2CF6
:10183000831685148312A210CB18A21422088500E7
:101840003A1D2F2C4B18272C83160511292C831693
:10185000051583122211CB18221522088500BA1D06
:101860003E2C4B18362C83168511382C8316851583
:101870008312A211CB18A21522088500391C4D2C09
:101880004B18452C83160512472C83160516831218
:101890002212CB18221622088500B91C5C2C4B188A
:1018A000542C83168512562C831685168312A21289
:1018B000CB18A21622088500391D6B2C4B18632CFF
:1018C00083160610652C8316061483122310CB187A
:1018D000231423088600B91D7A2C4B18722C83160A
:1018E0008611742C831686158312A311CB18A315A9
:1018F00023088600381C892C4B18812C831606126D
:10190000832C8316061683122312CB182316230862
:101910008600B81C982C4B18902C83168612922C9B
:10192000831686168312A312CB18A31623088600EB
:10193000381DA72C4B189F2C83160613A12C831639
:10194000061783122313CB18231723088600B81D0C
:10195000B62C4B18AE2C83168613B02C8316861724
:101960008312A313CB18A31723088600BA01B90169
:10197000B8013A1005183A14BA108518BA143A1179
:1019800005193A15BA108518BA143910051A391400
:10199000B910851AB914391106183915B9118619F3
:1019A000B9153810061A3814B810861AB814381138
:1019B000061B3815B811861BB8152508A60038086F
:1019C0008A1143208312A80039088A114320831208
:1019D000A9003A088A1143208312AA0008000A309D
:1019E0003B02031D352D2508A600DE01E201E301BF
:1019F0008A11942183124A1120184A158A154A1D0A
:101A0000202D620803191F2D5E1005185E14DE10CC
:101A1000861ADE145E11861B5E15DE11061BDE15AE
:101A20005E12061A5E165E088A1199218312DE1371
:101A3000E30A63088A15031D202DE203202DDE171B
:101A40008A11A8218312CA122018CA168A15CA1E22
:101A5000F82C8A11B6218312E500783065028A15C8
:101A6000031D412D0A30E200F82C3F30A60008008B
:101A7000831286183C2D382D8316061740308A11A4
:101A8000772908002508A60008002508A6002030B0
:101A9000A8005730A9006930AA007330AB0070303D
:101AA000AC003630AD003430AE003830AF002030FE
:101AB000B00008002508A60008002508A600203070
:101AC000A8003130A9002E30AA003230AB003730E8
:101AD000AC002030AD0008002708A60008008A11DD
:101AE000842083122508A6008A1171293F30A600A0
:101AF000080007309F00A21022088500A2112208CA
:101B0000850083160514851005118511051206142C
:101B10008615061686160617861740308A11772115
:101B20008312A31323088600831686138312C2012F
:101B3000831686138A117E2064308A11052083164D
:101B400086178A11842064308A1105208312C20A04
:101B5000033042028A15031D982D8A11A821831291
:101B6000C5102018C5148A15C518BA2D8A11AE20C3
:101B70008A15AD2D8A11B6218312C3007F3043052B
:101B8000A40024088A1123208312A5002330A60074
:101B9000463025028A150319CF2D0318D22D2508AA
:101BA000A600462E47302502031DD92D6F258A1524
:101BB000462E48302502031DE02D42258A15462E6B
:101BC00049302502031DE82D8A11A2268A15462ECA
:101BD0004A302502031DEF2D8B228A15462E4B30ED
:101BE0002502031DF62D76258A15462E4C3025023A
:101BF000031DFD2D53208A15462E4D302502031D51
:101C0000042E8B228A15462E4E302502031D0B2EE4
:101C10006C258A15462E50302502031D122E87236F
:101C20008A15462E51302502031D192E5A258A1574
:101C3000462E52302502031D212E8A11CF268A15E9
:101C4000462E53302502031D282E76258A15462E52
:101C500054302502031D2F2E45258A15462E563059
:101C60002502031D362E5D258A15462E5730250286
:101C7000031D3D2E53208A15462E58302502031D84
:101C8000452E8A11ED228A15462E762501308A11BD
:101C90004C20831225088A113A208312BB002608A3
:081CA0008A1199218A15AD2D6E
:02400E00423F2F
:00000001FF
